:107C0000112484B714BE81FFFDD085E080938100EC
:107C100082E08093C00088E18093C10096E0909359
:107C2000C20099E19093C400809360008EE080933D
:107C30006000259A86E028E13EEF91E030938500D0
:107C40002093840096BBB09BFECF1D9AA8958150CF
:107C5000A9F7C0E0D0E008E138E0F32EEE24E39489
:107C600045E0B42E51E1A52E13E0A7D0813491F464
:107C7000A4D0D82EAED082E8D81203C084E096D02B
:107C800092C0E1E8DE1203C084E090D08CC083E0B3
:107C90008DD089C0823419F484E1A7D084C08534A2
:107CA00019F485E0A2D07FC0853549F486D0C82F6D
:107CB00084D0D0E0D82BCC0FDD1F8BD074C086359C
:107CC00029F484E092D080E071D06DC0843609F050
:107CD0003FC073D072D0982E70D0C115F0E7DF0787
:107CE00038F4FE0117BFE895C12CDD24D39403C0FE
:107CF000C12CDD24D39461D0F60181936F019E12D3
:107D0000FACFC115F0E7DF0718F0FE0117BFE895BD
:107D100060D007B600FCFDCFFE01A0E0B1E08C9181
:107D200011962C91119790E0922B0C01E7BEE895EB
:107D3000112432961296A03881E0B80781F7FE012F
:107D4000B7BEE89507B600FCFDCFA7BEE8952BC0EF
:107D50008437B1F432D031D0982E2FD03AD0892C3C
:107D6000FE016F018FEFC81AD80A84911FD08A9440
:107D7000F6018110F6CF21969A94C90DD11D13C03A
:107D8000853741F426D08EE111D085E90FD08FE000
:107D90000DD009C0813531F400936000F09260008D
:107DA00018D001C016D080E101D05FCF9091C00003
:107DB00095FFFCCF8093C60008958091C00087FF97
:107DC000FCCF8091C00084FD01C0A8958091C600C1
:107DD0000895F3DF803239F088E18093600088E015
:107DE00080936000FFCF84E1E1CFCF93C82FE5DF20
:107DF000C150E9F7CF91EDCFE0E6F0E098E1908354
:107E000080830895E0E6F0E088E180831082EE2729
:047E1000FF270994AB
:027FFE00040479
:0400000300007C007D
:00000001FF
